:100000000C945D010C9485010C9485010C94850180
:100010000C9485010C9485010C9485010C94850148
:100020000C9485010C9485010C9477060C9443057F
:100030000C9485010C9485010C9485010C94850128
:100040000C9485010C9485010C9485010C94850118
:100050000C9485010C9485010C9485010C949F01EE
:100060000C9485010C9485010C9485010C948501F8
:100070000C9485010C9485010C9485010C948501E8
:100080000C9485010C9485010C9485010C948501D8
:100090000C9485010C9485010C9485010C948501C8
:1000A0000C9485010C9485010C948501A202A50293
:1000B000940298029E02C602C602C602A902AD02BE
:1000C000B102B702BB02C602C10200000002000971
:1000D0000F0000030401000C00000408020110409E
:1000E00080401020408040800802040180402010A1
:1000F000020110801020404004040404040304059D
:1001000002020202040302020202060606060606B4
:1001100004040202020400000000250028002B0055
:100120002E00310000000000240027002A002D00CE
:10013000300000C18081C112010002020000409C19
:10014000230C8000010102000112010002000000E6
:10015000409C230C80000101020001416461667231
:100160007569740046656174686572203332753450
:100170000004030904080B00020202010009040044
:100180000001020200000524001001052401010104
:10019000042402060524060001070581031000401F
:1001A00009040100020A00000007050202400000E5
:1001B0000705830240000000000000000000002A44
:1001C0002B280000000000000000000000000000DC
:1001D000000000000000002C9EB4A0A1A2A434A640
:1001E000A7A5AE362D3738271E1F20212223242510
:1001F00026B333B62EB7B89F8485868788898A8BC5
:100200008C8D8E8F909192939495969798999A9BB6
:100210009C9D2F3130A3AD350405060708090A0B54
:100220000C0D0E0F101112131415161718191A1B96
:100230001C1DAFB1B0B500090402000103000000AD
:100240000921010100012265000705840340000126
:1002500005010902A1010901A10085010509190192
:100260002903150025019503750181029501750586
:10027000810305010930093109381581257F750889
:1002800095038106C0C005010906A1018502050785
:1002900019E029E7150025017501950881029501EE
:1002A0007508810395067508150025650507190071
:1002B00029658100C0009F07F20811241FBECFEFFF
:1002C000DAE0DEBFCDBF11E0A0E0B1E0EEE5F2E1A3
:1002D00002C005900D92A832B107D9F721E0A8E23B
:1002E000B1E001C01D92A739B207E1F712E0CAEBF5
:1002F000D2E004C02297FE010E942909C63BD10723
:10030000C9F70E9437030C942D090C94000061E09A
:100310008DE00C94C70261E08DE00E94000368EE5E
:1003200073E080E090E00E940C0260E08DE00E94AB
:10033000000368EE73E080E090E00C940C021F92E2
:100340000F920FB60F9211242F933F938F939F9389
:10035000AF93BF938091290190912A01A0912B0125
:10036000B0912C013091280126E0230F2D3720F485
:100370000296A11DB11D05C029E8230F0396A11DFA
:10038000B11D209328018093290190932A01A09305
:100390002B01B0932C0180912D0190912E01A09101
:1003A0002F01B09130010196A11DB11D80932D0147
:1003B00090932E01A0932F01B0933001BF91AF9184
:1003C0009F918F913F912F910F900FBE0F901F9093
:1003D00018953FB7F89480912D0190912E01A0912E
:1003E0002F01B091300126B5A89B05C02F3F19F011
:1003F0000196A11DB11D3FBF6627782F892F9A2F27
:10040000620F711D811D911D43E0660F771F881FCC
:10041000991F4A95D1F70895CF92DF92EF92FF92FC
:10042000CF93DF936B017C010E94E901EB01C114C2
:10043000D104E104F10489F00E94E1060E94E9017F
:100440006C1B7D0B683E734090F381E0C81AD108A5
:10045000E108F108C851DC4FEACFDF91CF91FF905E
:10046000EF90DF90CF900895789484B5826084BD3A
:1004700084B5816084BD85B5826085BD85B58160A8
:1004800085BDEEE6F0E0808181608083E1E8F0E008
:100490001082808182608083808181608083E0E837
:1004A000F0E0808181608083E1E9F0E0808182601A
:1004B0008083808181608083E0E9F0E080818160D9
:1004C0008083E1ECF0E080818460808380818260C1
:1004D0008083808181608083E3ECF0E080818160B3
:1004E0008083E0ECF0E0808182608083E2ECF0E0E9
:1004F000808181608083EAE7F0E08081846080838E
:1005000080818260808380818E7F8083808180680B
:100510008083089590E0FC013197EF30F105B0F54C
:10052000EA5AFF4F0C942709809180008F7703C00F
:10053000809180008F7D809380000895809180005D
:10054000877FF9CF84B58F7702C084B58F7D84BD56
:100550000895809190008F7707C0809190008F7DE3
:1005600003C080919000877F8093900008958091D0
:10057000C0008F7703C08091C0008F7D8093C00042
:1005800008958091C200877F8093C2000895CF9321
:10059000DF9390E0FC01E652FF4F2491FC01E8500C
:1005A000FF4F8491882349F190E0880F991FFC0147
:1005B000EC5DFE4FA591B4918A5E9E4FFC01C59102
:1005C000D4919FB7611108C0F8948C912095822333
:1005D0008C93888182230AC0623051F4F8948C9104
:1005E000322F309583238C938881822B888304C09B
:1005F000F8948C91822B8C939FBFDF91CF910895BB
:100600000F931F93CF93DF931F92CDB7DEB7282FA1
:1006100030E0F901E653FF4F8491F901E652FF4FB4
:100620001491F901E850FF4F04910023C9F0882389
:1006300021F069830E948A026981E02FF0E0EE0FC9
:10064000FF1FEA5EFE4FA591B4919FB7F8948C917D
:10065000611103C01095812301C0812B8C939FBF32
:100660000F90DF91CF911F910F91089508950E94EF
:1006700034020E94360381E391E00E94C5060E9485
:100680008701C0E0D0E00E948B012097E1F30E9437
:100690000000F9CF4091350150913601209133018E
:1006A0003091340142175307B4F49091E8009570EB
:1006B000E1F39091E80092FD19C08093F1008091E0
:1006C00035019091360101968F739927892B19F482
:1006D0008EEF8093E800809135019091360101966C
:1006E000909336018093350181E0089580E008956C
:1006F000CF92DF92FF920F931F93CF93DF931F92BE
:10070000CDB7DEB7082F162F862F880F8E5F9983FF
:100710000E944A0383E00E944A03F02EC02E998172
:10072000D92E8C2D8F19811778F4F60184910E94AF
:100730004A03082F80E00E944A038023FFEFCF1A6C
:10074000DF0A8111EECF01C081E00F90DF91CF91E0
:100750001F910F91FF90DF90CF900895615030F07E
:100760002091F100FC0120830196F8CF84E680936C
:10077000380108952FB7FC012083F89467706093C7
:10078000E9000895CF93DF931F92CDB7DEB7682FAE
:10079000CE0101960E94BA038091F20099819FBF19
:1007A0000F90DF91CF910895FF920F931F93CF93F6
:1007B000DF9300D0CDB7DEB7F62E8A0190913701D6
:1007C000992311F057FF03C08FEF9FEF2AC0682FC6
:1007D000CE0101967A830E94BA038091F20090E0E4
:1007E000A8017A81801791070CF4AC01EF2DF72F47
:1007F000F40E84E6FE1631F0809338019091F100FA
:100800009193F8CF4115510521F08091F200882392
:1008100021F089818FBFCA0104C08BE68093E80074
:10082000F8CF0F900F90DF91CF911F910F91FF9014
:100830000895CF93DF931F92CDB7DEB741E050E02C
:10084000BE016F5F7F4F0E94D403019719F4898125
:1008500090E002C08FEF9FEF0F90DF91CF9108954E
:10086000CF93DF931F92CDB7DEB7682FCE010196ED
:100870000E94BA039091E800892F807295FF04C00E
:100880009091F20080E4891B99819FBF0F90DF91C6
:10089000CF9108956F927F928F929F92AF92BF9265
:1008A000CF92DF92EF92FF920F931F93CF93DF933C
:1008B0001F92CDB7DEB7782E7B01C42EB52E809166
:1008C0003701882369F0042F152F8AEFD82E872D42
:1008D0008072982E9AE3A92E872D8074882E11C0DD
:1008E0008FEF9FEF56C0872D0E943004682E811134
:1008F0000CC0DA94A9F361E070E080E090E00E941F
:100900000C020115110579F73BC0282F30E00217C2
:1009100013070CF4602E672DCE0101960E94BA03D6
:100920008091E80085FF29C0262D30E0021B130BC3
:10093000992039F06A948FEF6816B1F01092F100A7
:10094000F9CFF701862D77FE07C0815058F09491BA
:100950009093F1003196F9CF815020F091919093CE
:10096000F100FACFE20EF31E8091E80085FF0EC081
:100970000115110511F4811009C089818FBFC1CF04
:1009800084E6809339018C2D9B2D03C0A092E80052
:10099000F4CF0F90DF91CF911F910F91FF90EF90C7
:1009A000DF90CF90BF90AF909F908F907F906F908F
:1009B00008951092E900109236011092350190933B
:1009C0003401809333010895CF92DF92FF920F9309
:1009D0001F93CF93DF9300D0CDB7DEB7F82E8A01F7
:1009E0006B0101151105B1F0F601F7FE02C084910B
:1009F00001C0808149835A830E944A030150110932
:100A0000FFEFCF1ADF0A49815A818111EACF8FEFB8
:100A10009FEF01C0CA010F900F90DF91CF911F91FE
:100A20000F91FF90DF90CF9008951F93CF93DF93A6
:100A30001F92CDB7DEB7162F2091E80022FFFCCF22
:100A4000612F79830E94AE038BEF8093E800812FA2
:100A50007981972F0F90DF91CF911F910895CF93B8
:100A6000DF931F92CDB7DEB71982CE0101960E94A7
:100A70003F07CE0101960E94DA07898190E00F902E
:100A8000DF91CF9108951F920F920FB60F9211240C
:100A9000EF92FF920F931F932F933F934F935F9388
:100AA0006F937F938F939F93AF93BF93EF93FF9336
:100AB000CF93DF93CDB7DEB76297DEBFCDBF109285
:100AC000E9008091E80083FFEBC068E0CE010A9660
:100AD0000E94AE0382EF8093E8009A8597FF05C0DD
:100AE0008091E80080FFFCCF03C08EEF8093E80088
:100AF000892F807609F0B9C08B85811105C01092CD
:100B0000F1001092F100C5C0282F2D7F213009F48B
:100B1000C0C0853049F48091E80080FFFCCF8C850F
:100B200080688093E300B5C0863009F076C02D85DB
:100B3000E888F988223071F580E090E02A8B0E94E5
:100B4000D9040E942F0599E08E010F5F1F4FF80115
:100B5000392F11923A95E9F799832A892A8391E0EE
:100B60009E8390E898879AEF99872091350130917C
:100B70003601275F3F4F3C832B838D83C7010E9443
:100B8000D90449E050E0B80180E00E94E4040E94EA
:100B90002F057FC0C7012A8B0E94D9042A892232DF
:100BA00041F482E290E00E94E507892B09F071C0D0
:100BB00074C0213069F488899989089711F42093C9
:100BC000320180913201811118C069E471E01AC0CC
:100BD000233009F062C08C85882391F0823021F4A3
:100BE0006CE084E691E006C0813009F056C068E010
:100BF0008BE591E00E9478034AC067E371E002C090
:100C000061E771E06115710509F447C0FB0144918A
:100C100050E080E80E94E4043CC0873009F43DC005
:100C2000883021F481E08093F10033C0893089F568
:100C3000937099F5E3E3F1E081E021E096E380939E
:100C4000E9002093EB0034913093EC009093ED0099
:100C50008F5F3196853099F78EE78093EA00109286
:100C6000EA008C858093370114C0888999890E9495
:100C7000D9048E85811105C0CE010A960E944A07CB
:100C800006C0823051F4CE010A960E940D088823D6
:100C900021F08EEF8093E80003C081E28093EB00A7
:100CA00062960FB6F894DEBF0FBECDBFDF91CF9135
:100CB000FF91EF91BF91AF919F918F917F916F9134
:100CC0005F914F913F912F911F910F91FF90EF9066
:100CD0000F900FBE0F901F9018958093E9008091A0
:100CE000F200882319F08AE38093E80008951F92A8
:100CF0000F920FB60F9211242F933F934F935F9350
:100D00006F937F938F939F93AF93BF93EF93FF93D3
:100D10008091E1001092E10083FF0FC01092E90082
:100D200091E09093EB001092EC0092E39093ED0031
:100D30001092370198E09093F00082FF15C083E095
:100D40000E946D0680913901882329F08091390134
:100D500081508093390180913801882329F0809156
:100D60003801815080933801FF91EF91BF91AF918D
:100D70009F918F917F916F915F914F913F912F91B3
:100D80000F900FBE0F901F9018951092370181E0C1
:100D90008093D70080EA8093D80082E089BD09B4AF
:100DA00000FEFDCF61E070E080E090E00E940C0268
:100DB00080E98093D8008CE08093E2001092E000FC
:100DC00008950895CF93DF931F92CDB7DEB769835F
:100DD000DC01ED91FC910280F381E02D41E050E0D7
:100DE000BE016F5F7F4F09950F90DF91CF910895FE
:100DF000CF93DF93EC018C859D8597FF05C082E042
:100E00000E9419049D878C878C859D85DF91CF91E9
:100E1000089583E00C946D06FC018485958597FD0B
:100E200006C082E00E94C20390E00196089582E02D
:100E30000E94C20390E00895FC018485958597FD8A
:100E400005C02FEF3FEF35872487089582E00C948B
:100E50001904CF93DF93EC0180910701882331F0CF
:100E600083E00E944A041816190634F081E090E0ED
:100E70009B838A8380E090E0DF91CF910895FC010D
:100E800020812E5F208342E450E065E771E080E836
:100E90000C94E404FC0181819081913A59F48132EF
:100EA00009F03CC047E050E060E071E080E00E9463
:100EB000E40443C0913291F5803239F467E070E088
:100EC00080E091E00E94150506C0823209F035C02D
:100ED0008281809307018091000190910101A0918E
:100EE0000201B0910301803B9440A105B105C1F41A
:100EF0008091070180FD14C087E797E79093010870
:100F0000809300082BE088E190E00FB6F894A89554
:100F1000809360000FBE209360000FC080E00895B2
:100F200088E10FB6F89480936000109260000FBEC5
:100F3000A895109201081092000881E0089510927F
:100F40003D0110923C0188EE93E0A0E0B0E0809378
:100F50003E0190933F01A0934001B09341018EE088
:100F600091E090933B0180933A018FEF9FEF909334
:100F70004701809346010895FF920F931F93CF93EB
:100F8000DF93EC01F62EE881F9810480F581E02DF4
:100F900009958C01E881F9810680F781E02D6F2D9C
:100FA000CE010995C8019927DF91CF911F910F912B
:100FB000FF900895FC0120812F5F208349E150E0DC
:100FC00067E372E080E80C94E40445E650E060E5F5
:100FD00072E080E80C94E404EF92FF920F931F9369
:100FE000CF93DF931F92CDB7DEB789838B017A0150
:100FF00041E050E0BE016F5F7F4F84E00E944A04F1
:10100000A701B80184E40E944A040F90DF91CF91B8
:101010001F910F91FF90EF900895FC0191818081C5
:10102000813A31F481E0913091F0933089F411C02C
:10103000813271F49B3021F482818093090105C0D3
:101040009A3031F482818093080181E008950895F7
:1010500080E0089548E050E082E00C94EC07CF93E4
:10106000DF93DC01683818F0E8E7E60F25C0E62FCB
:10107000F0E067FF11C0E058F10981E090E001C0A5
:10108000880FEA95EAF714969C911497982B14967A
:101090009C931497E0E010C0E954FE4FE491EE23D6
:1010A00009F440C0E7FF08C014968C911497826041
:1010B00014968C931497EF7716968C9116978E173B
:1010C00041F117968C9117978E1719F118968C91FC
:1010D00018978E17F1F019968C9119978E17C9F001
:1010E0001A968C911A978E17A1F01B968C911B97CC
:1010F0008E1779F080E090E0ED01C80FD91F2E81A6
:10110000211102C0EE8305C0019686309105A1F73A
:1011100009C0BD016C5F7F4FCD010E942A0881E0AC
:1011200090E008C081E090E013969C938E93129714
:1011300080E090E0DF91CF910895683818F0E8E7FB
:10114000E60F25C0E62FF0E067FF12C0E058F10976
:1011500021E030E001C0220FEA95EAF72095DC019A
:1011600014963C911497322314963C93E0E00FC000
:10117000E954FE4FE491EE2329F1E7FF08C0DC01BA
:1011800014962C9114972D7F14962C93EF7720E0D2
:1011900030E0EE2351F0DC01A20FB31F16964C9104
:1011A00016974E1302C016961C922F5F3F4F2630A3
:1011B000310579F7BC016C5F7F4F0E942A0881E0FE
:1011C00090E0089580E090E00895FC011682178277
:1011D00010861186128613861482BC016C5F7F4FC5
:1011E0000C942A081092960110928D0110928C0195
:1011F0008EE191E090938B0180938A010895CF92C4
:10120000DF92EF92FF920F931F93CF93DF936C01C6
:101210007A01EB01E60EF71E00E010E0CE15DF05C7
:1012200061F06991D601ED91FC910190F081E02D82
:10123000C6010995080F191FF1CFC801DF91CF91A1
:101240001F910F91FF90EF90DF90CF900895EE0FD8
:0E125000FF1F0590F491E02D0994F894FFCF54
:10125E0000E1000000000000010100000000E206B5
:10126E0029070C071C07F806090700000000BC0739
:08127E00FF082F089D08E50898
:00000001FF
